:020000040000FA
:0400000068303A2802
:040004000034003490
:08000800A000030EA100831209
:1000100005191128831601178312B2308100B1012E
:100020002C2883160113831203140B190310A80D37
:10003000A90DAA0DAB0DAC0DAC16FF302C02031DA3
:100040002C28FA302B02031D2C2832152A08AF0069
:100050002908AE002808AD008B100B11210E83007B
:06006000A00E200E0900B5
:0C007400203084008001840A80300402E7
:10008000031C3C285E2183160C30850587018312F2
:10009000850187010730990000309A0010308316DF
:1000A0008E008312603083168F0083120030831617
:1000B000910000008312C830831681008312313012
:1000C0009000003083168C00831210308B00BD1B13
:1000D0006F2885196F286400851D6B2886213D1CBB
:1000E00072287B2181018E018F010B118B100B1067
:1000F0008C018B178A20321996204021B40B882856
:10010000031085190314BA0DF0303A020319EE20DA
:10011000AC217A2864003310B10A311F9528AC0154
:10012000AB01AA01A901A801B101080032110130F7
:10013000B7008B132030370783169B001C141A0856
:100140008312A4001030370783169B001C141A0872
:100150008312A300A6000230A606003037078316DC
:100160009B001C141A088312A200A7000130A706E6
:100170008B17331CC12822090339A200A309A40943
:10018000A50924082F02031DE82823082E02031DB9
:10019000D62822082D02031DE82801303702031D4E
:1001A000D6283E18D6283E143F146F2126082E026A
:1001B000031DE82827082D02031DE8280130370217
:1001C000031DE7283E1CE7283E103F147221E82853
:1001D000B70A023037020318080099280130B60028
:1001E000B400B500B70085018701B2137A218A20D7
:1001F000B40B0729031085190314BA0DF0303A0225
:1002000003192F29B50B07299630B5003B21321D64
:10021000F7283211331C11292D090339AD00AE091D
:10022000AF092F1CF7282D0830020319F7282D08D5
:10023000B0002E1EF7288B1320303707BC002F0884
:10024000BB00492110303707BC002E08BB004921F4
:1002500000303707BC002D08BB0049218B178501F2
:100260008701B70AB6010130B50002303702031C1E
:10027000F7287B2108000130370203197621080096
:100280003F1C08003F101030BC003E08BB00492155
:1002900008008B133B0883161C159A0083123C0838
:1002A00083169B0055309D00AA309D009C1464006D
:1002B0009C1857291C1183128B17080083160030D5
:1002C0009B001C141A088312BD003D1C08008316F5
:1002D00010309B001C141A088312BE000800013065
:1002E000BE00080087010530D40008000508333A35
:1002F00085000800080001303E020319802908002B
:100300000130D40056150730D3000800B601B401FF
:10031000B5013D1C8E29BD01BD149029BD013D14C0
:100320003D08B600640094299529962997299829B3
:100330003330B51B8500B51F8501B40B9229B50B71
:1003400092290310B60CB608031D92290030BC0098
:100350003D08BB00492108008F08031908008E01E1
:100360008F01D0080319FC29D00FC929561805168A
:10037000D618851656190514D6198514D60158189D
:100380000512D818851258190510D8198510D801EA
:10039000FC295008D10056180516D618851656198E
:1003A0000514D619851451080E020318E3295818AC
:1003B0000512D818851258190510D8198510FF3064
:1003C0005002031908008F08031D08008A205108F5
:1003D0000E02031CE32956180512D6188512561969
:1003E0000510D619851058180516D81885165819ED
:1003F0000514D8198514080000305302031D152A6E
:100400003E180D2A051A58140130051AD000851A15
:10041000D8140130851AD00008000130D4005614D9
:100420000130D0000130D3000800051A1B2A5614F1
:10043000851AD8141D2AD61458140130D000D40BB4
:10044000080001305302031D2F2AD6150530D400B1
:100450000230D3003E180800D601D3010800023054
:100460005302031D412A56158714D8150330D400B2
:100470000330D3003E1808008701D601D301D815F8
:10048000080003305302031D512A87140715033057
:10049000D4000430D3003E1808008701D30158155A
:1004A000080004305302031D622A8714071507143D
:1004B0000330D4000530D3003E1808008701D30173
:1004C0005815080005305302031D742A87140715B8
:1004D000071487160330D4000630D3003E180800F6
:1004E0008701D3015815080006305302031D872ADF
:1004F000871407150714871607160330D400073032
:10050000D3003E1808008701D301581508000730B2
:100510005302031D9B2A8714071507148716071615
:1005200087150130D4000730D3003E18080087013A
:0C053000D301581508000030D30008006B
:084000000700030007000100A6
:02400E00CC33B1
:10420000010078007A007C007E007B0079007F004E
:104210007D007A0078007E007C00FF00FF00FF0038
:104220000000F200F600FA00FE00F200F600FA00CC
:10423000FE00F200F600FA00FE00FF00FF00FF00A3
:10424000010005000500050005000900090009003E
:1042500009000D000D000D000D00FF00FF00FF0024
:10426000FF00FF00FF00FF00FF00FF00FF00FF0056
:10427000FF00FF00FF00FF00FF00FF00FF00FF0046
:10428000FF00FF00FF00FF00FF00FF00FF00FF0036
:10429000FF00FF00FF00FF00FF00FF00FF00FF0026
:1042A000FF00FF00FF00FF00FF00FF00FF00FF0016
:1042B000FF00FF00FF00FF00FF00FF00FF00FF0006
:1042C000FF00FF00FF00FF00FF00FF00FF00FF00F6
:1042D000FF00FF00FF00FF00FF00FF00FF00FF00E6
:1042E000FF00FF00FF00FF00FF00FF00FF00FF00D6
:1042F000FF00FF00FF00FF00FF00FF00FF00DD00E8
:00000001FF
